:020000020000FC
:0200040064D1C5
:0200080062D1C3
:02000C0060D1C1
:020010005ED1BF
:020014005CD1BD
:020018005AD1BB
:02001C0058D1B9
:0200200056D1B7
:0200240054D1B5
:0200280052D1B3
:02002C0050D1B1
:020030004ED1AF
:020034004CD1AD
:020038004AD1AB
:02003C0048D1A9
:0200400046D1A7
:0200440044D1A5
:0200480042D1A3
:02004C0040D1A1
:020050003ED19F
:020054003CD19D
:020058003AD19B
:02005C0038D199
:0200600036D197
:0200640034D195
:0200680032D193
:02006C0030D191
:020070002ED18F
:020074002CD18D
:020078002AD18B
:02007C0028D189
:0200800026D187
:0200840024D185
:0200880022D183
:02008C0020D181
:020090001ED17F
:020094001CD17D
:020098001AD17B
:02009C0018D179
:0200A00016D177
:0200A40014D175
:0200A80012D173
:0200AC0010D171
:0200B0000ED16F
:0200B4000CD16D
:0200B8000AD16B
:0200BC0008D169
:0200C00006D167
:0200C40004D165
:0200C80002D163
:0200CC0000D161
:0200D000FED060
:0200D400FCD05E
:0200D800FAD05C
:0200DC00F8D05A
:1000E000F6D000200010FFFF39000A0041546D6572
:1000F00067613132383007FF3E72782D62756600D5
:1001000000008200082F10911002E0E0F2E0E10F01
:10011000F31D008313951F7010931002899199911C
:100120000C9404F006FF6973722D72787B0000F066
:1001300045F0C600A9F0C2F045F00300AAFD3EF06C
:10014000A20073FA810025F000F045F0970045F019
:100150003200A1F445F0000245F0160065F1E9F423
:1001600025F006FF72782D627566920000F0D100CE
:100170003EF0B70045F01102A9F0C2F045F00002D0
:10018000AEF1A9F0D5F040F245F00F0024F245F0B1
:1001900011029EF025F007FF72783F2D6275660010
:1001A000B10000F06BFA45F01102A9F045F0100221
:1001B000A9F024F125F007FF74782D706F6C6C00A6
:1001C000CB0000F0EF003EF0E20045F0C6009EF0EC
:1001D00025F008FF74783F2D706F6C6CDB0000F029
:1001E0006BFA45F0C000A9F045F0200024F225F09C
:1001F00004FF75627272E90080F0CA00CEFBD8FB82
:1002000006FF2B7573617274F80000F045F09800DA
:1002100045F0C1009EF045F0060045F0C2009EF09A
:10022000FC00C2F00AF345F0C5009EF045F0C400A2
:100230009EF0A40025F008FF31772E726573657477
:10024000000122019A938A936C9A7498E0E8F7E08F
:100250003197F1F71FB7F894749A6C98E0E0F1E0E9
:100260003197F1F78CB184FF9FEF1FBF6C987498A2
:10027000E0E8F6E03197F1F7892F0C9404F007FFDE
:1002800031772E736C6F74001B01460174986C9A61
:100290001FB7F894E8E1F0E03197F1F7889487957B
:1002A00010F4749A6C98E4E2F0E03197F1F70CB135
:1002B00004FD8068ECECF0E03197F1F7749A6C98EB
:0E02C000E8E0F0E03197F1F71FBF0C9404F076
:040000000C9474FAEE
:1002CE000A920FB60A920F900F900A94B02CFF93D9
:1002DE00EF93E2E1F2E00694E00DF31D008003944B
:1002EE000082EF91FF9109900FBE0990089502FFD1
:1002FE006D2B3F0100F092FD2FF425F003FF756486
:10030E002A007E0100F0C2F010F1F1F1EAF0D5F012
:10031E0007F1F1F1F2F0AEF125F004FF756D6178A1
:10032E00850100F07FF56DF13EF09E01D5F0EAF00B
:10033E0025F004FF756D696E940100F07FF578F17C
:10034E003EF0AA01D5F0EAF025F000F045F000806D
:10035E0024F22BF13EF0B501B1FD25F05CF125F054
:10036E000AFF6E616D653E666C616773A00100F0F9
:10037E00E2F345F000FF24F225F006FF6E65776587
:10038E007374B70153F04B0206FF6C61746573749E
:10039E00C40153F04F0208FF28637265617465292A
:1003AE00CB0100F0CEF92F03C2F0C90178F592F01F
:1003BE001403C90192F025F001005C00D20100F097
:1003CE00B5F901F198F592F025F001002800E3014E
:1003DE0000F045F02900A1F988F525F007FF636FBD
:1003EE006D70696C6500EC0100F007F1C2F0C5FBA1
:1003FE0010F1E2F3060225F001FF2C00F50100F0EA
:10040E00C8F584F3C8F540F2B3FBC9F525F0030037
:10041E005B275D00030200F024F81C0225F00700A4
:10042E006C69746572616C000E0200F0FB0145F0A0
:10043E00060225F00800736C69746572616C160211
:10044E0000F0FB0187F795F725F000F0C8F5FB01EA
:10045E00FFFF25F000F071FBC8F5D5F084F325F011
:10046E0000F0C8F525F000F071FB060225F005003E
:10047E00616865616400210200F0FB0134F02C021A
:10048E0025F0020069663E0200F0FB013EF02C02F0
:10049E0025F00400656C7365480200F0FB0134F032
:1004AE002C02D5F0310225F004007468656E5002FE
:1004BE0000F0310225F00500626567696E005B028F
:1004CE0000F0370225F005007768696C650062025E
:1004DE0000F04B02D5F025F0060072657065617470
:1004EE006A0200F08C025F0225F00500756E7469D9
:1004FE006C00730200F045F03EF006023A0225F061
:10050E000500616761696E007C0200F0FB0134F04A
:10051E003A0225F00200646F870200F0FB01ACF294
:10052E00370265F1EF0225F004006C6F6F709102D7
:10053E0000F0FB01DAF2D60225F005002B6C6F6F8E
:10054E0070009B0200F0FB01CBF2D60225F00500F5
:10055E006C6561766500A40200F0FB01E5F24302D2
:10056E00EF0225F003003F646F00AE0200F0FB01C6
:10057E00C5024B029402D5F0EF0225F000F07FF594
:10058E00AAFDC2F010F13EF0CD0288F507F10EF291
:10059E0025F007FF656E646C6F6F7000B90200F096
:1005AE003A02E302CAF03EF0DF025F0234F0D802F4
:1005BE0025F002FF6C3ED00200F002038AF08AF0B2
:1005CE0045F0FEFF020376F225F002FF3E6CE002DC
:1005DE0000F0B6FD020376F202038AF092F025F0E7
:1005EE0003FF6C703000EC0280F07E00CEFBD8FB77
:1005FE0002FF6C70F70253F0510206FF63726561E1
:10060E007465FF0200F0D8013803FB0160F025F09D
:10061E0006FF686561646572040300F0C8F510F1A9
:10062E0010F1C2F039F13EF02603C2F045F000FFA2
:10063E002DF299F707F170F3060207F125F045F058
:10064E00F0FF5BF807FF776C73636F7065000F0345
:10065E002DFC7A00CEFBD8FB06FF72657665616CC9
:10066E00290300F0C90178F58AF0CAF03EF0430381
:10067E00C9018AF0D5F04CF325F00500646F65735F
:10068E003E00330300F0FB015C03FB010E94FB0103
:10069E00510325F09A938A93CB0101967F916F9126
:1006AE00BF93AF93DB010C9404F000F007F1C90186
:1006BE0078F58AF070F398FC84F325F001FF3A0088
:1006CE00440300F0D8017303EAF025F007FF3A6EF9
:1006DE006F6E616D6500650300F0C8F5C2F0D00164
:1006EE0092F0FB0100F0880325F001003B006D0342
:1006FE0000F0FB0125F09003380325F001FF5D00AB
:10070E007C0300F0B1FD65F592F025F001005B0071
:10071E00850300F065F165F592F025F008FF76612E
:10072E00726961626C658D0300F0D9F5A703B6FDA1
:10073E00E2F525F008FF636F6E7374616E749503B6
:10074E0000F0D8013803FB0153F0060225F004FF38
:10075E0075736572A10300F0D8013803FB0166F0D2
:10076E00060225F007007265637572736500AE03AD
:10077E0000F0D0018AF0060225F009FF696D6D6563
:10078E00646961746500B90300F06D0470F3C2F022
:10079E00E2F345F0FF7F24F2D5F084F325F0060056
:1007AE005B636861725DC40300F0FB0145F004F900
:1007BE00060225F0060061626F727422D60300F005
:1007CE00DBF4FB01F80325F005FF61626F72740024
:1007DE00E10300F05CF15BF806FF3F61626F72743B
:1007EE00EB0300F0F2F03EF0FE03BAF7F00388F5EB
:1007FE0025F009FF6765742D737461636B00F30355
:10080E0000F0C2F078F5D5F070F3C2F010F165F19A
:10081E00D5F0C5023EF01E04ACF2BDF246F272F502
:10082E00E0F0AEF170F3D5F05CF1CBF2140488F584
:10083E0007F125F009FF7365742D737461636B0006
:10084E00000400F0E0F032F13EF0300445F0FCFF21
:10085E005BF87FF54CF3D5F065F1C5023EF03D0433
:10086E00ACF278F590F54CF3DAF23804EAF025F0B4
:10087E0009FF6D61702D737461636B00210400F0CC
:10088E00C2F078F5D5F070F372F589FDC5023EF031
:10089E006204ACF2BDF270F3D5F010F119F12FF045
:1008AE00CAF03EF05E0407F1EAF0E5F225F007F13A
:1008BE00B6FDCBF25104EAF065F125F00BFF67654A
:1008CE00742D63757272656E74003F0400F045F00E
:1008DE00840070F325F009FF6765742D6F726465EF
:1008EE007200650400F045F08800070425F009FF4A
:1008FE006366672D6F7264657200720453F0880030
:10090E0007FF636F6D70617265007E048E04BF9386
:10091E00AF938C0189919991DC01899199919C01F8
:10092E0089919991FC01ED90F190EF1451F40A9593
:10093E0019F02A95C1F701C02A95022B11F48827C8
:10094E0002C08FEF00C0982FAF91BF910C9404F0AE
:10095E0007FF6E66613E6C666100870400F08CFCDA
:10096E0040F215F2AEF125F00BFF7365742D637531
:10097E007272656E7400AF0400F045F084004CF3A3
:10098E0025F008FF776F72646C697374BB0400F016
:10099E00D1F565F1E0F04CF3C2F078F5B3FBD2F58A
:1009AE0025F00EFF666F7274682D776F72646C6936
:1009BE007374C80453F0860009FF7365742D6F724B
:1009CE0064657200D80400F045F08800280425F014
:1009DE000FFF7365742D7265636F676E697A65724A
:1009EE007300E30400F045F09A00280425F00FFF91
:1009FE006765742D7265636F676E697A65727300D1
:100A0E00EF0400F045F09A00070425F004FF636F31
:100A1E006465FE0400F0D8013803C8F5C5FB060274
:100A2E0025F008FF656E642D636F64650D0500F09B
:100A3E00FB010C94FB0104F025F008FF286D617298
:100A4E006B657229180580F0A600CEFBD8FB080056
:100A5E00706F7374706F6E65240500F0CEF9E6FA50
:100A6E00F1FAC2F010F1C5FBC5FBE2F32FF007F16E
:100A7E00C5FBE2F3060225F00BFF6170706C747516
:100A8E00726E6B6579002E0500F0050193F47EFB06
:100A9E00FCF787F70A00466F7274686475696E6FAB
:040AAE00BAF725F07E
:020000021000EC
:10E00000BF93AF93DB011196B21499F4FD0155272C
:10E01000EE0FFF1F551F5BBF679177911196FB01B4
:10E020005527EE0FFF1F551F5BBF07911791F80192
:10E0300009949A938A938B2D9927BB246CEB74EFE8
:10E04000EECF04FF65786974430526F0AF91BF9168
:10E05000DBCF07FF657865637574650021F030F0EC
:10E06000BC0189919991DBCF35F0FD015527EE0F69
:10E07000FF1F551F5BBFA791B791C6CF3FF0982BED
:10E080008991999191F31196BFCF46F09A938A9313
:10E09000FD015527EE0FFF1F551F5BBF879197911D
:10E0A0001196B2CF53F09A938A93FB01319655277C
:10E0B000EE0FFF1F551F5BBF87919791A5CF60F0B3
:10E0C0009A938A93CB0101969FCF66F09A938A9395
:10E0D000FB0131965527EE0FFF1F551F5BBF879140
:10E0E0009791840D951D90CF07FF2876616C75651B
:10E0F000290029F000F0D8013803FB0180F025F059
:10E100000E945103C2F0C5FBE2F32FF025F001FF9E
:10E11000400074F08BF0FC018191919175CF01FF6B
:10E12000210087F093F0FC0189919991918380837C
:10E130008991999169CF02FF63218FF09FF0FC01D3
:10E14000899199918083899199915ECF02FF634073
:10E150009BF0AAF0FC019927808156CF02FF407501
:10E16000A6F000F013F3AEF18AF025F002FF21755E
:10E17000AEF000F013F3AEF192F025F003FF6475FA
:10E180007000B6F0C3F09A938A933ECF04FF3F64C9
:10E190007570BEF0CBF0082F092B11F09A938A937B
:10E1A00033CF04FF73776170C6F0D6F08C0189918C
:10E1B00099911A930A9328CF04FF6F766572D1F074
:10E1C000E1F09A938A938A819B811ECF04FF647247
:10E1D0006F70DCF0EBF08991999116CF03FF726FAD
:10E1E0007400E6F0F3F08C012991399189919991AD
:10E1F0003A932A931A930A9307CF03FF6E6970002C
:10E20000EEF002F1229600CF02FF723EFDF008F11F
:10E210009A938A938F919F91F7CE02FF3E7204F1F9
:10E2200011F19F938F9389919991EECE02FF7240E5
:10E230000DF11AF19A938A938F919F919F938F93E7
:10E24000E3CE02FF3C3E16F100F0AAFD2BF125F0D3
:10E2500002FF303D21F12CF1982BD1F530C002FFA7
:10E26000303C28F133F197FD2AC032C002FF303E26
:10E270002FF13AF1821593055CF151F120C003FFB3
:10E2800064303E0036F144F18215930589919991ED
:10E2900082059305ECF0E1F012C003FF64303C000E
:10E2A0003FF152F1229697FD0C945FF10C9468F1C6
:10E2B00004FF747275654DF15DF19A938A938FEF47
:10E2C0009FEFA2CE01FF300058F166F19A938A9336
:10E2D000C1019ACE02FF753C62F16EF1299139912C
:10E2E00082179307A8F3A1F3EACF02FF753E6AF104
:10E2F00000F0D5F06DF125F001FF3C0075F180F1E3
:10E3000029913991281739071CF7D9CF01FF3E0011
:10E310007CF18AF12991399128173907CCF2C1F2A1
:10E32000CECF04FF6C6F673286F196F1FC0199271E
:10E3300080E18A9522F0EE0FFF1FD8F765CE9A95FF
:10E3400063CE01FF2D0091F1A5F109911991081BF0
:10E35000190BC80159CE01FF2B00A1F1AFF10991B2
:10E360001991800F911F50CE02FF6D2AABF1B8F1C9
:10E370008C01899199919C0131027001209FC0010B
:10E380003003F308900DE11CF31C1203F308900D09
:10E39000E11CF31C9A938A93C70136CE06FF756D74
:10E3A0002F6D6F64B4F1D4F17C01299139910991F9
:10E3B000199140E15527000F111F221F331F551FD0
:10E3C0002E153F05520518F003952E193F094A9561
:10E3D00089F73A932A93C80117CE03FF756D2A0077
:10E3E000CEF1F2F18C0189919991809FF001222761
:10E3F0003327909FF00D211D331D819FF00D211DAE
:10E40000331D919F200D311DCF019A938A93C9012D
:10E41000FBCD06FF696E76657274EDF10FF28095A3
:10E420009095F2CD02FF322F09F216F2959587955D
:10E43000EBCD02FF322A12F21DF2880F991FE4CDB4
:10E4400003FF616E640019F225F20991199180238E
:10E450009123DACD02FF6F7220F22EF20991199109
:10E46000802B912BD1CD03FF786F72002AF238F206
:10E470000991199180279127C7CD02FF312B33F2E3
:10E4800041F20196C1CD02FF312D3DF247F20197D5
:10E49000BBCD07FF3F6E65676174650043F200F016
:10E4A00032F13EF054F259F625F006FF6C736869BC
:10E4B000667449F25BF2FC018991999131971AF0E7
:10E4C000880F991FFBCFA0CD06FF72736869667431
:10E4D00055F26AF2FC018991999131971AF096955B
:10E4E0008795FBCF91CD02FF2B2164F277F2FC01DF
:10E4F0008991999120813181820F931F808391832B
:10E500008991999181CD03FF7270400073F288F276
:10E510009A938A938DB79EB777CD03FF72702100CF
:10E5200083F292F22FB7F8948DBF9EBF2FBF8991CF
:10E5300099916ACD03FF737040008DF29FF29A9318
:10E540008A93CE0161CD03FF737021009AF2A8F285
:10E55000EC018991999158CDADF229913991E0E87A
:10E560003E0F821B930B3F932F939F938F93899121
:10E5700099914ACD01FF6900A3F2BEF29A938A9362
:10E580008F919F91EF91FF91FF93EF939F938F93C3
:10E590008E0F9F1F39CDCCF2EF91FF91E80FF91F3D
:10E5A000899199911BF0FF93EF935FCD0F911F918C
:10E5B00011962ACDDBF2EF91FF913196BBF3F3CFA9
:10E5C00006FF756E6C6F6F70BAF2E6F21F910F91D5
:10E5D0001F910F9119CD06FF636D6F76653EE0F2D6
:10E5E000F1F2BF93AF93E991F991A991B991092FF4
:10E5F000082B41F0E80FF91FA80FB91F1E911293C5
:10E600000197E1F7AF91BF9189919991FDCC02FFFC
:10E610003E3CEBF20BF3092F982F802FF5CC03FF34
:10E620007570400007F314F39A938A93C201ECCCFF
:10E6300003FF757021000FF31DF32C01899199914F
:10E64000E3CC03FF316D730018F326F3E0EAFFE03B
:10E650003197F1F7D9CC03FF323E720021F330F34A
:10E66000FC01899199919F938F93FF93EF938991E7
:10E670009991CACC03FF32723E002BF33FF39A9379
:10E680008A93EF91FF918F919F919A938A93CF01F3
:10E69000BBCC02FF21653AF34DF3FC0189919991BE
:10E6A0002FB7F89428D000B5081709F00BD0319691
:10E6B00022D000B5091711F0892F04D02FBF8991FE
:10E6C0009991A2CCF999FECF07B700FDFDCFF2BD1D
:10E6D000E1BD80BDFA9AF99A089502FF406549F3B9
:10E6E00071F32FB7F894FC0106D080B5319603D0B2
:10E6F00090B52FBF89CCF999FECFF2BDE1BDF89A54
:10E70000089502FF21696DF32DFCA400CEFBD8FB18
:10E7100009FF2821692D6E727777290081F390F324
:10E720001FB71F93F8949C0189919991AF93BF9360
:10E73000CF93DF9309D0DF91CF91BF91AF918991B2
:10E7400099911F911FBF60CC10D0E094F0948E215E
:10E750009F21982B19F0F90102E023D0F90104E080
:10E7600020D0F90100E11DD00895F901E078FF7F84
:10E77000EF01A0E8B0E0FE015527EE0FFF1F551F87
:10E780005BBF47915791FE01E217F30711F00A01B1
:10E7900002C07A010C01002704D02196119759F785
:10E7A0000895F999FECF17B710FDFDCF5527EE0F4D
:10E7B000FF1F551F5BBF016007BFE895089502FF6B
:10E7C000406988F3E3F3FC015527EE0FFF1F551F47
:10E7D0005BBF8791979118CC03FF6E3E7200DFF309
:10E7E000F1F3FC01082F899199919F938F930A95DA
:10E7F000D1F7EF93FF938991999106CC03FF6E7245
:10E800003E00ECF303F49A938A93FF91EF910E2F5D
:10E810008F919F919A938A930A95D1F7CF01F4CB68
:10E8200003FF64322A00FEF315F409911991000FD9
:10E83000111F881F991F1A930A93E6CB03FF6432B6
:10E840002F0010F423F40991199195958795179548
:10E8500007951A930A93D8CB02FF642B1EF430F469
:10E8600029913991E990F99049915991240F351FD7
:10E870008E1D9F1D3A932A93C7CB02FF642D2CF463
:10E8800041F429913991E990F99049915991421BAC
:10E89000530BE80AF90A5A934A93C701B5CB07FF0D
:10E8A00064696E76657274003DF456F409911991AD
:10E8B00080959095009510951A930A93A5CB02FF29
:10E8C000752E4FF400F065F144F725F003FF752E27
:10E8D00072005FF400F065F1D5F04DF725F00DFF03
:10E8E00073686F772D776F72646C6973740066F468
:10E8F00000F045F07EF4D5F071FC25F000F08CFCC2
:10E90000BAF7FCF75CF125F005FF776F72647300CE
:10E910006FF400F045F08A0070F378F425F004FFFE
:10E920002B696E7484F494F478946ECB04FF2D6993
:10E930006E748FF49BF4F89467CB04FF696E7421B6
:10E9400096F400F045F00000AEF14CF325F004FF22
:10E95000696E74409DF400F045F00000AEF170F374
:10E9600025F008FF696E742D74726170A7F4B8F415
:10E97000B82E8991999148CB00F0ABF42FF0C1F4F7
:10E9800025F0C2F401D040CB189504FF7069636B89
:10E99000B1F400F040F272F59EF2AEF18AF025F08B
:10E9A00002002E22C5F400F0DBF4FB01BAF725F0DB
:10E9B00002007322D0F400F045F02200A1F965F5C1
:10E9C0008AF03EF0E4F4270225F004FF66696C6CDF
:10E9D000D8F400F0F2F0F2F0CAF03EF0F6F489FD5F
:10E9E000ACF2C2F0BDF29EF0DAF2F1F4EAF025F0FA
:10E9F0000BFF656E7669726F6E6D656E7400E5F47F
:10EA000053F0820009FF776F72646C69737473004E
:10EA1000000000F045F0080025F004FF2F7061644D
:10EA200002F500F09EF29EF5A4F125F005FF2F6897
:10EA30006F6C64000DF500F09EF5D9F5A4F125F09A
:10EA40000AFF666F7274682D6E616D6516F500F0D1
:10EA500087F70700616D666F7274680025F007FF25
:10EA600076657273696F6E0020F500F045F0410025
:10EA700025F003FF637075002FF500F045F0750079
:10EA8000E6F725F008FF6D63752D696E666F39F541
:10EA900000F045F0710025F005FF2F7573657200D9
:10EAA00042F500F045F02C0025F005FF665F63702D
:10EAB0007500F8F400F045F0002445F0F40025F06E
:10EAC00005FF73746174650055F553F0530204FF3C
:10EAD0006261736560F566F00C0005FF63656C6C40
:10EAE000730067F51DF205FF63656C6C2B006DF517
:10EAF00079F5029689CA04FF3264757073F500F0E7
:10EB0000E0F0E0F025F005FF3264726F70007BF5F5
:10EB100000F0EAF0EAF025F004FF7475636B83F50A
:10EB200000F0D5F0E0F025F003FF3E696E008CF5B3
:10EB300066F0180003FF7061640094F500F0D9F5E9
:10EB400045F02800AEF125F004FF656D69749AF573
:10EB50002DFC0E00F6FB02FC05FF656D69743F009D
:10EB6000A4F52DFC1000F6FB02FC03FF6B65790099
:10EB7000ACF52DFC1200F6FB02FC04FF6B65793F3F
:10EB8000B5F52DFC1400F6FB02FC02FF6470BDF528
:10EB900080F07400CEFBD8FB05FF656865726500E8
:10EBA000C5F580F07800CEFBD8FB04FF6865726580
:10EBB000CCF580F07600CEFBD8FB05FF616C6C6F66
:10EBC0007400D5F500F0D9F5AEF1B3FBDAF525F018
:10EBD00003FF62696E00DDF500F0B6FD6BF592F0A3
:10EBE00025F007FF646563696D616C00E8F500F06E
:10EBF00045F00A006BF592F025F003FF6865780098
:10EC0000F1F500F045F010006BF592F025F002FFF1
:10EC1000626CFDF553F0200007FF7475726E6B6532
:10EC2000790007F62DFC8000CEFBD8FB04FF2F6D8A
:10EC30006F640CF61BF69C0109911991412F432733
:10EC400017FF04C0109500950F5F1F4F37FF04C0DA
:10EC5000309520952F5F3F4FEE24FF1851E1001FA4
:10EC6000111F5A9539F447FF04C0109500950F5FA6
:10EC70001F4F0BC0EE1CFF1CE21AF30A20F4E20E39
:10EC8000F31E8894ECCF0894EACFFA92EA92C80176
:10EC9000BBC905FF752F6D6F640016F600F010F10B
:10ECA00065F107F1D3F125F006FF6E6567617465C4
:10ECB00049F600F00EF240F225F001FF2F0054F665
:10ECC00000F01AF601F125F003FF6D6F64005DF6A8
:10ECD00000F01AF6EAF025F003FF6162730064F6B3
:10ECE00000F0C2F04FF225F003FF6D696E006CF684
:10ECF00000F07FF589F13EF07EF6D5F0EAF025F0E0
:10ED000003FF6D61780074F600F07FF57FF13EF04F
:10ED10008AF6D5F0EAF025F006FF77697468696E27
:10ED200080F600F0E0F0A4F110F1A4F107F16DF12C
:10ED300025F007FF746F7570706572008CF600F037
:10ED4000C2F045F0610045F07B0091F63EF0ABF675
:10ED500045F0DF0024F225F007FF746F6C6F7765D4
:10ED6000720099F600F0C2F045F0410045F05B00FA
:10ED700091F63EF0BEF645F020002DF225F003FF9F
:10ED8000686C6400ACF653F0550204FF686F6C6465
:10ED9000BFF600F0C3F6C2F08AF046F2C2F010F1FE
:10EDA000D5F092F007F19EF025F002FF3C23C5F666
:10EDB00000F09EF5C3F692F025F001FF2300D5F692
:10EDC00000F06BF58AF05DF7F2F045F00900E0F035
:10EDD0007FF13EF0EEF645F00700AEF145F0300071
:10EDE000AEF1C9F625F002FF2373DDF600F0E0F680
:10EDF0007FF52DF22BF13EF0F7F625F002FF233ED2
:10EE0000F3F600F088F5C3F68AF09EF5E0F0A4F181
:10EE100025F004FF7369676EFEF600F032F13EF0F4
:10EE200014F745F02D00C9F625F003FF642E72009B
:10EE300009F700F010F190F5FFFCD8F6F6F6F2F0C5
:10EE40000DF701F707F1E0F0A4F105F815F825F04A
:10EE500002FF2E7215F700F010F192FD07F119F77D
:10EE600025F002FF642E28F700F065F119F7FCF792
:10EE700025F001FF2E0031F700F092FD34F725F068
:10EE800003FF75642E0039F700F065F14DF7FCF7CC
:10EE900025F004FF75642E7240F700F010F1D8F6EB
:10EEA000F6F601F707F1E0F0A4F105F815F825F002
:10EEB00006FF75642F6D6F6449F700F010F165F17E
:10EEC00019F1D3F107F1D5F010F1D3F107F125F0E5
:10EED00006FF64696769743F58F700F09FF6C2F057
:10EEE00045F0390089F145F0000124F2AEF1C2F09D
:10EEF00045F0400189F145F0070124F2A4F145F005
:10EF00003000A4F1C2F06BF58AF06DF125F000F04D
:10EF100019F1E6F707F1E0F040F215F2AEF140F238
:10EF200010F125F002FF732C68F700F0C2F099F79A
:10EF300025F000F00602C2F015F290F51CF2A4F1E3
:10EF400010F165F1C5023EF0ACF7ACF2C2F08AF008
:10EF5000060278F5DAF2A6F707F139F13EF0B3F7D9
:10EF6000C2F0A9F00602EAF025F005FF6974797095
:10EF7000650092F700F0C2F015F290F51CF2A4F1D2
:10EF800010F165F1C5023EF0CEF7ACF2C2F0E2F34B
:10EF9000C2F0DBF7D7F740F2DAF2C6F707F139F142
:10EFA0003EF0D5F7C2F0E2F3DBF7EAF025F000F02F
:10EFB0000AF3DBF725F000F045F0FF0024F2A8F596
:10EFC00025F006FF69636F756E74B5F700F0C2F047
:10EFD00040F2D5F0E2F325F002FF6372E1F700F0B2
:10EFE00045F00D00A8F545F00A00A8F525F005FF4D
:10EFF000737061636500ECF700F00AF6A8F525F080
:10F0000006FF737061636573F7F700F065F184F6CE
:10F01000C2F03EF00FF8FCF746F234F008F8EAF0E0
:10F0200025F004FF7479706500F800F089FDC502D1
:10F030003EF020F8ACF2BDF2A9F0A8F5DAF21BF828
:10F0400025F001FF270011F800F0CEF9E6FAF1FAF9
:10F05000C2F064FBAAFDD5F0E2F345F099FBAAFDEE
:10F060002DF23EF036F845F0F3FF5BF8EAF025F0BC
:10F0700007FF68616E646C65720021F866F00A0033
:10F0800005FF63617463680038F800F09EF210F1C8
:10F090003EF88AF010F187F23EF892F02FF007F177
:10F0A0003EF892F007F1EAF065F125F005FF74688B
:10F0B000726F770040F800F0C2F02BF13EF062F87A
:10F0C000EAF025F03EF88AF091F207F13EF892F06E
:10F0D00007F1D5F010F1A7F2EAF007F125F005FFEE
:10F0E00063736B69700056F800F010F1C2F03EF0E7
:10F0F00083F8E0F0A9F019F1AAFD3EF083F8B1FD24
:10F10000BFF934F076F807F1EAF025F005FF6373F4
:10F1100063616E006FF800F010F1E0F0C2F0A9F04A
:10F1200019F1AAFD2BF13EF0A0F8D5F046F2D5F08A
:10F13000E0F032F12BF13EF0A0F840F234F08EF81E
:10F1400001F1E0F0A4F107F1EAF025F006FF6163B8
:10F150006365707486F800F0E0F0AEF146F2E0F01E
:10F16000B9F5C2F0ECF82BF13EF0DEF8C2F045F054
:10F170000800AAFD3EF0CEF8EAF0F2F07FF589F142
:10F1800010F1F2F0F2F007F13EF0CCF8E4F846F2BC
:10F1900010F1E0F007F1980134F0DCF8C2F00AF663
:10F1A0007FF13EF0D5F8EAF00AF6C2F0A8F5E0F0FB
:10F1B0009EF040F2E0F0A40134F0B0F8EAF001F182
:10F1C000D5F0A4F1EFF725F000F045F00800C2F00B
:10F1D000A8F5FCF7A8F525F000F0C2F045F00D0009
:10F1E000AAFDD5F045F00A00AAFD2DF225F006FF94
:10F1F000726566696C6CA6F82DFC1A00F6FB02FCC1
:10F2000004FF63686172F7F800F0CEF9EAF0A9F044
:10F2100025F006FF6E756D62657200F900F06BF502
:10F220008AF010F152F910F165F952F907F12DF257
:10F2300010F1C2F02BF13EF025F988F507F1EAF064
:10F2400007F16BF592F065F125F02FF365F165F1AB
:10F250003EF383F9CAF03EF047F9B1FDAAFD3EF056
:10F260003EF9A9F045F02E00AAFD3EF03FF907F166
:10F270003EF03BF90CFDB6FD34F04DF9EAF088F5AF
:10F2800007F1EAF007F16BF592F065F125F088F5EA
:10F2900007F13EF04CF959F6B1FD07F16BF592F02C
:10F2A0005CF125F000F0E0F0A9F045F02D00AAFD9A
:10F2B000C2F010F13EF05EF9B1FDBFF907F125F0A3
:10F2C00060F00A00100002000A0000F0E0F0A9F06F
:10F2D00045F02300A4F1C2F065F145F0040091F679
:10F2E0003EF07BF960F9AEF1E2F36BF592F0B1FD1F
:10F2F000BFF934F07CF9EAF025F007FF3E6E756D3A
:10F300006265720009F900F0C2F03EF09BF9E0F08E
:10F31000A9F06DF72BF13EF08FF9EAF025F010F12E
:10F3200030FD6BF58AF0890107F1810130FDB1FDF7
:10F33000BFF934F084F925F005FF70617273650040
:10F340007DF900F010F1B5F998F58AF0BFF907F1F1
:10F350008BF8C2F040F298F576F2B1FDBFF925F0D6
:10F3600006FF736F757263659CF92DFC1600F6FB42
:10F3700002FC07FF2F737472696E6700B0F900F02A
:10F38000F2F0E0F0AEF1F2F0F2F0A4F125F00AFFB5
:10F3900070617273652D6E616D65B9F900F00AF6E2
:10F3A000D2F925F000F010F1B5F998F58AF0BFF91F
:10F3B00019F174F807F18BF87FF5AEF1B5F9EAF0C1
:10F3C000A4F198F592F025F007FF66696E642D7838
:10F3D0007400C7F900F045F0F6F945F088004604DE
:10F3E0002BF13EF0F5F988F565F125F000F010F10C
:10F3F0007FF507F13FFCC2F03EF003FA10F101F196
:10F4000001F107F15CF125F000F087F70300206FB0
:10F410006B00BAF725F003FF2E6F6B00E4F92DFCAB
:10F420001C00F6FB02FC00F087F702003E20EFF71D
:10F43000BAF725F006FF2E72656164790BFA2DFC90
:10F440002000F6FB02FC00F087F70400203F3F207D
:10F45000BAF76BF58AF010F1F7F53CF798F58AF0FA
:10F460003CF707F16BF592F025F006FF2E657272FE
:10F470006F721AFA2DFC1E00F6FB02FC04FF717578
:10F48000697435FA00F0FB02020392F0A3FAA7F2C6
:10F49000B0FA91F2900365F58AF02BF13EF051FA43
:10F4A0001FFAFCF83EF063FA45F0C9FA45F8CAF0D5
:10F4B0003EF063FAC2F045F0FEFF7FF13EF061FAE4
:10F4C0003AFA34F043FA0FFA34F04BFA05FF706160
:10F4D000757365003EFA2DFC5702E2FBECFB04FF5E
:10F4E000636F6C6466FA74FAA4B622243324BB24D6
:10F4F00024BEE0E0F2E02192E030E9F7F232D9F701
:10F50000E9E5F2E02F010FEF0DBF048311E21EBF0A
:10F510001583CFEAC683D1E2D783A6E9BAEF0C946C
:10F5200004F004FF7761726D6FFA00F07BFD45F027
:10F5300099FB45F06BFA0DFC900312F642FA03FFBB
:10F540007370300091FA80F00600F6FB02FC02FFB7
:10F5500073709FFA66F0080003FF72703000A7FA1C
:10F5600000F0B4FA8AF025F066F0040005FF646547
:10F5700070746800ACFA00F0A3FA9EF2A4F115F2E0
:10F5800046F225F009FF696E746572707265740049
:10F59000B6FA00F0CEF9C2F03EF0DAFAE6FAF1FA85
:10F5A00065F58AF03EF0D5FAC5FBE2F32FF071FB6A
:10F5B00034F0CAFA88F525F010FF666F7274682D72
:10F5C0007265636F676E697A6572C2FA80F07C005B
:10F5D000CEFBD8FB09FF7265636F676E697A6500C1
:10F5E000DCFA00F045F0FCFAD5F046042BF13EF0D1
:10F5F000FBFA88F564FB25F000F0F2F0F2F07FF5FD
:10F600002FF3F2F02FF03EF3F2F0C2F064FBAAFD0C
:10F610003EF00DFBEAF065F125F001F101F15CF13E
:10F6200025F006FF64743A6E756DEAFA60F099FB96
:10F630001C021C0207FF64743A646E756D0011FBB6
:10F6400060F099FBA2FDA2FD07FF7265633A6E753B
:10F650006D001AFB00F00EF93EF036FBB1FDAAFD7D
:10F660003EF034FB16FB25F020FB25F064FB25F073
:10F6700008FF7265633A66696E6424FB00F0EAF97C
:10F68000C2F02BF13EF047FBEAF064FB25F04EFBA5
:10F6900025F005FF64743A78740038FB60F052FB83
:10F6A00056FBA2FD00F0EAF02FF025F000F032F159
:10F6B0003EF05CFB060225F02FF025F007FF647496
:10F6C0003A6E756C6C0049FB60F068FB68FB68FB88
:10F6D00000F045F0F3FF5BF806FF3F737461636B66
:10F6E0005EFB00F0BBFA32F13EF079FB45F0FCFF27
:10F6F0005BF825F003FF766572006CFB00F027F5E0
:10F70000BAF7FCF76BF58AF035F5F7F592FDD8F608
:10F71000E0F645F02E00C9F6F6F601F715F86BF5A0
:10F7200092F0FCF73DF5BAF725F004FF6E6F6F70AD
:10F730007AFB00F025F006FF756E7573656495FB26
:10F7400000F09EF2D9F5A4F125F00200746F9BFB46
:10F7500000F024F89BFD65F58AF03EF0B9FBFB0153
:10F76000B3FB060225F000F007F1C2F0C5FB10F173
:10F77000E2F3C2F0C5FBC5FBE2F32FF025F007FF73
:10F78000692D63656C6C2B00A5FB00F040F225F041
:10F7900007FF4564656665724000BFFB00F0E2F359
:10F7A00070F325F007FF4564656665722100C8FBAC
:10F7B00000F0E2F34CF325F007FF526465666572D2
:10F7C0004000D2FB00F0E2F38AF025F007FF52641C
:10F7D000656665722100DCFB00F0E2F392F025F033
:10F7E00007FF5564656665724000E6FB00F0E2F3D2
:10F7F00013F3AEF18AF025F007FF55646566657274
:10F800002100F0FB00F0E2F313F3AEF192F025F0EB
:10F8100006FF646566657221FCFB00F09BFDC2F08B
:10F82000C5FBC5FBE2F32FF025F006FF64656665B6
:10F83000724008FC00F09BFDC2F0C5FBE2F32FF024
:10F8400025F007FF286465666572290015FC00F045
:10F85000D8013803FB012DFC25F00E945103C2F0B2
:10F86000C5FBE2F32FF02FF025F00FFF73656172F7
:10F8700063682D776F72646C6973740021FC00F00B
:10F8800010F165F145F054FC07F171FCC2F02BF169
:10F890003EF04EFC88F5EAF065F125F0C2F098FCE8
:10F8A000D5F0BE01AC0125F000F010F1EAF07FF5D3
:10F8B00019F18CFCA2FC3EF062FC07F1EAF065F164
:10F8C0005CF125F088F507F165F125F011FF747200
:10F8D0006176657273652D776F72646C69737400FD
:10F8E00035FC00F070F3C2F03EF082FC7FF52FF3A0
:10F8F000D5F02FF03EF3F2F03EF082FCB504E2F3D7
:10F9000034F073FC88F525F00BFF6E616D653E7376
:10F910007472696E670066FC00F0E6F745F0FF0060
:10F9200024F225F007FF6E66613E6366610084FC89
:10F9300000F0B50440F225F008FF69636F6D706157
:10F94000726592FC00F010F1E0F007F124F13EF056
:10F95000ADFC88F5EAF05CF125F0D5F065F1C50263
:10F960003EF0D2FCACF2E0F08AF0D5FCE0F0E2F33D
:10F97000D5FCC2F045F000016DF13EF0C3FCD5F0BE
:10F9800045F0FF0024F224F13EF0CAFC88F55CF15A
:10F99000E5F225F040F2D5F078F5D5F045F002001B
:10F9A000CBF2B3FC88F565F125F000F0C2F045F02C
:10F9B000FF0024F2B2F6D5F00AF345F0FF0024F27E
:10F9C000B2F60AF32DF225F001FF2A009CFC00F0AC
:10F9D000B7F1EAF025F001FF6A00E4FC00F087F2DD
:10F9E00045F00700AEF18AF087F245F00900AEF16C
:10F9F0008AF0AEF125F004FF64616273EBFC00F065
:10FA0000C2F032F13EF005FD0CFD25F007FF646EFB
:10FA1000656761746500FBFC00F055F4B1FD65F1AC
:10FA20002FF425F005FF636D6F76650006FD18FD68
:10FA3000BF93AF93E991F991A991B991092F082B3F
:10FA400021F01D9111930197E1F7AF91BF91899139
:10FA500099910C9404F005FF32737761700012FDE8
:10FA600000F0F2F010F1F2F007F125F00AFF7265F4
:10FA700066696C6C2D7469622BFD00F059FD45F0D0
:10FA80005A00ABF85FFD92F065F198F592F05CF1E9
:10FA900025F00AFF736F757263652D74696236FD18
:10FAA00000F059FD5FFD8AF025F003FF74696200E4
:10FAB00049FD53F0850204FF2374696255FD53F03C
:10FAC000DF0206FF65653E72616D5BFD00F065F16A
:10FAD000ACF2E0F070F3E0F092F078F5D5F078F564
:10FAE000D5F0DAF269FD88F525F008FF696E6974D2
:10FAF0002D72616D61FD00F045F0A80013F345F033
:10FB0000220015F266FD25F006FF626F756E6473C4
:10FB100075FD00F0E0F0AEF1D5F025F003FF733E87
:10FB2000640084FD00F0C2F032F125F005FF3E6272
:10FB30006F6479008EFD41F20800326C6974657261
:10FB4000616C96FD00F0D5F01C021C0225F001FF4F
:10FB50003D009CFD00F0A4F12BF125F001FF3100E8
:10FB6000A7FD53F0010001FF3200AEFD53F002008B
:0AFB700002FF2D31B3FD53F0FFFF3B
:00000001FF
